:020000040000FA
:040000000000C32F0A
:08000800FB00030EFD000408DB
:10001000FC0083120313831314207C0884007D0EDC
:100020008300FB0E7B0E09000C191B288B1825285A
:100030008C1A502808000C114C194E2CD0080319AA
:100040000800CC0A8316981608008B102008820737
:100050002E28342838283C28412808000517A217E4
:100060002A08A300A00A0800A30B0800A00A0B128C
:10007000A21B0800A00A0B1605130830A300A00A53
:10008000080021088400800D03180517031C0513C0
:10009000A30B0800A003A10AA20B0800A0010800FE
:1000A00098184E2C18194E2C0A30CB004C19D12C14
:1000B0004C08033982077A2C942C9D2C922C083CF6
:1000C000031882070034E634DC34D234C834BE343A
:1000D000B434AA34A03403398207CC2E382FCC2E66
:1000E000C12E0F3982070134043407340E34023430
:1000F0000534083400340334063409340F340A3428
:100100000B340C340D348207BD29AD29A52999295A
:10011000902945298207372A1E2A152A0F2AF429F1
:10012000F1291F3982077E3430346D347934333409
:100130005B345F3470347F347B3477341F340D3458
:100140003D344F344734173410340E3405341D34E5
:100150001C343E3467344E34463401344034083461
:10016000193415340034132684234E2472150330B9
:10017000C920AF00FF30BC007B30C2001530B10099
:10018000B330B0008B170B160030C9200319452976
:10019000302983169B001C141A0883120800B32010
:1001A000F220D320D028A21FD828F11BA82E382F48
:1001B0000C1A6D2CCC1B662C4C1AB02CBF1B7B2947
:1001C000C308031D3F2E711BED28AE08031D982B9D
:1001D00070190D2CF119322C08007108D03A03194E
:1001E0006F2908000B1D0800073081070B11CB0891
:1001F0000319FD28CB0BFD28CC17BC0803190529D2
:10020000BC0B05291430BC00E425C20803190D29D4
:10021000C20B0D297D30C200431730083104031989
:1002200022290130B002031CB10330083104031D40
:1002300022290330B100E830B0000830AE000317C7
:10024000261303133208330403192F290130B20295
:10025000031CB30332083304031D2F297015080053
:100260001030AA001E302E27143039278515F214BD
:100270007214F211FF30C40024309A260430B30007
:10028000D230B2008030F100080014304527382702
:100290008511F2107210F2150830F50075088B23E5
:1002A0000330840701308000F50B4E290F30C40065
:1002B0000C309A26B201B3010030F100080015306D
:1002C000AA003330C40010309A265030F1000800E4
:1002D0003330C40020309A264030F1000800E30893
:1002E000031908003330C4001C309A26B201B30150
:1002F000C030F1000800BF133F080F39F11B8929F6
:10030000711B89290A3A03193029013A03195F2917
:100310000800093C0318F42A063E711B8A2883282A
:1003200071180800F11908007108803A03196F2943
:1003300008007118A229F1190800630803190800C0
:100340009023F12B71107015080071180800F1113D
:10035000F123E4080319F12308007118B329701E72
:10036000F115701208000330E21BE2066205031D5E
:100370002C3003192830E2179A2E711C08007110D6
:10038000701540307427770878040319080078083E
:10039000E1007708E000610DE00DE113B2230319DD
:1003A000E129E3008B23840A00083039303A03192D
:1003B000E929FC308005E204620980046308E40056
:1003C000080008309A260530B300DC30B200333024
:1003D000EE290930B300C430B2005530C4007011AA
:1003E0000800F11B452930297108503A0319682982
:1003F000303A03196829203A03196129803A031910
:100400003A29F039903A03196129303A03196829D9
:10041000203A03196829803A03196F2908007108E6
:100420001F39023A03194A2A080071081F39023A93
:1004300003194D2A103903196C2A080071089F39D5
:10044000013A0319C02A033A0319C02A013A0319D1
:10045000C02A133A0319DB2A013A03199C2A7C3972
:10046000143A0319B62A0C3A0319B42A0800710881
:100470001F39013A03197A2A033A03197A2A013AF1
:1004800003197A2AFC39043A03198A2A0C3A031907
:100490007E2A0800B803B7016C2AB80AB7016C2A93
:1004A000403074277708031D632A780803196B2AE4
:1004B000F11F642A013A03196B2A103A03196B2AB7
:1004C000033A03196B2A7808FF3EB800031CF703B0
:1004D0007708B700013E08007108F0390238F100D2
:1004E00037080339B700F7003808013EF800031851
:1004F000F70A852A71105022031908007108F03993
:100500000438F1003908F800F7018D277908C00098
:100510007A080D2BAB227108F0390838F1003A083F
:100520000739C900CA01BA19CA0AC9170B30C7006E
:100530001F30C800C31708004030742778087704BC
:1005400003196129382B4908BA00CA08031DBA15D6
:100550003A167110080040307427F708031D7A2AF4
:100560007808B90071100800A322B72AAB227108DD
:10057000F039403A0319322B803A0319562B45299A
:100580007110502203190800C6227E2AF115083086
:10059000BB00B9013708B4003808B5003B03083880
:1005A000BA006A230310F0190314B90DBB0BCA2A51
:1005B000F11139080800F7011C30B800B701C62254
:1005C000B80120390319EA2A1030B800C6223F3991
:1005D000F700B80AC622F8007704031961293330FE
:1005E000C4008D2781266529093CF300711FFA2A72
:1005F000F119202B7118032B7114711FF111E201F5
:10060000C00173080D2BE2130F30C005C00EC10EE0
:100610004105C004F03041057304C100FF30C4003F
:1006200040308126C813C913CA13711F0800711AFC
:1006300008000F30C0050C3071190D30C7000800DC
:10064000083A0319312B013A0319312B893AC906AB
:10065000C90003192D2BCA012F2B0130CA06C3175D
:10066000C91708003708B4003808B5006A2368299C
:1006700040307427F530BA00B501780D770D003E93
:1006800003194C2BBA151030B500B4017708C038E7
:10069000B9006A231130B500B4017808B9006A23A3
:1006A000F1151C30B500B4016A2361293708B40084
:1006B0003808B500E03077238830C4001E30332678
:1006C00063088B2303193A29013084078017D2303D
:1006D000F10008007030772325260A302E272726C0
:1006E0000530512725260A302E273827272EB40417
:1006F000F1197E2B3908B6000C30822B3A08E0380D
:10070000B6000830B40408000830F50075039123E2
:10071000F50B862B0800FF3E5F208400003E08009A
:10072000FF3E8C23031908008001840A8001080021
:10073000AE032E088C230319080080080319080053
:100740008003031D0800840A00083039303A031D75
:10075000080080127015E4080319F12308002F081F
:100760008000080060086104031900348039031D0B
:1007700000340830F500F30175038C23840A801AD5
:10078000C52B7508F300001ED32B013084076108C8
:100790000006031DD32B0430840760080006031DE8
:1007A000D32B75080800F50BBC2B73080319003414
:1007B0008B230A30F500840784038001F50BDC2BC2
:1007C000840A23308000840A610880000430840792
:1007D00060088000FD3084070130800073087015C8
:1007E000080070150830F500E408031DF5036408DF
:1007F0008C23031DFD2BE401F72B840A00083039FC
:100800000319052C303A031D0A2CE40AF50BF72BCB
:10081000E4010B2CE40A6408080070117108803AA6
:10082000031D0800FF30C400C813C913CA136408AD
:10083000E30003192D2C8B23840A001AC917801A90
:10084000CA17840A0008F800043084070008F7007B
:10085000F80DF70CF80C8D27812E1F3033261A3037
:10086000CA0008005F08031908008B2303194A2CEB
:10087000DF00033E84000008F800F7017026C9136A
:10088000CA135F08043E8400801E4A2C4708803942
:100890001A38C700DF01FF30C400080083160C11AE
:1008A0008C1298128312061518121A081A081816B4
:1008B00098175230CD00CC01CF01D001CB010C11E3
:1008C00083168C168312C713C3170800CC1A4E2C3C
:1008D0004C196C2C592C08004E2C4C1D08004C183F
:1008E00008004E08840000089900CE0AD00B0800CA
:1008F000CC0A08001A08D100DE00E039A03A03193A
:100900008B2C403A03198E2C603A0319892CCB01A9
:10091000080001308C2C0330CF00CC0ACC0AC7175A
:10092000C31708001A0808001A08DE060E3A031D4D
:10093000592C0C30CF00CC0A0800CF0BA72C1A087A
:100940005E06FF3A031D592CCC0A4C1608004D08D0
:1009500084001A088000DE06801B592CCD0A08008E
:100960004C125108A03A0319E02C013A0319E22C69
:10097000033A0319E42C173A0319DE2C0A3A031937
:10098000F22C053A0319FD2C013A0319FB2C543AB9
:100990000319342D6D3A0319D92C013A0319DB2CB4
:1009A000592C4D0884001A080006CD0ACF0B080008
:1009B00008004521592C711F3021592C0130E62C9B
:1009C0000330E62C0430E62C0730E62CDE0052081B
:1009D000DF008B230319592CAF235E0884075308CB
:1009E0008000592C5208E0005308E100B223003E79
:1009F000031D702DCA2D5208702D520803191A2D8F
:100A000053080319242D5206031DCA2D52088B23A7
:100A10000319CA2DAF23840A000830390319CA2DDF
:100A2000303A0319CA2D8004520864060319F123D1
:100A30005208702D64080319CA2DD2008B23840A32
:100A400000168016F123FB2C52088B230319CA2DA4
:100A5000840A000830390319CA2D303A031980126C
:100A60005208E4007015702D52088B23031D4A2D87
:100A700052087B3A031D402D831720308400502DEF
:100A8000073A031D492D53080C39043A031D7F30E2
:100A9000CB2DC82D540859040319CA2DAF23840A3D
:100AA00053088000840A54088000840A5508800096
:100AB000840A56088000840A58088000840A59086D
:100AC0008000840A5A088000840A5B088000840A37
:100AD0005C0880008313E4080319F1230130CB2D57
:100AE000D300DE008B23031D8F2D5308031D862D9D
:100AF000D401D501D601D701D901DA01DB014D308E
:100B0000DC00DE064230DD00DE06BD2D7B3A031D33
:100B10008D2D831720308400902D7B3AC82D840AB8
:100B200000087F39D400DE06840A00087F39D5002A
:100B3000DE06840A00087F39D600DE06840A000833
:100B40007F39D700DE06840A00087F39D900DE0627
:100B5000840A00087F39DA00DE06840A00087F393B
:100B6000DB00DE06840A00087F39DC00DE06840A2A
:100B700000087F39DD00DE068313E730D100DE0692
:100B80007208D800DE060E30D200DE06DE09D62D51
:100B90007F30CB2D0301D300D40051087F39D20020
:100BA000D406B430D100D406D4090430CF00D0002C
:100BB0005130CD00013ECE0051089900D0030C11F8
:100BC00083160C1583120800BE08031DBE03031D07
:100BD00008000430BD00BD030508FC393D04850054
:100BE0000000060E0F390F3A031DFB2DBD08031D33
:100BF000EB2D3F13002E3F1B022E0326C038BF00F3
:100C00000230BE000800F300003073180E2E013EC3
:100C1000F3180E2E013E73190E2E013E0310BD0D6A
:100C2000BD0D3D0471280330C6000B30C5005826A9
:100C30000030C6000930C5005826FF30C400C3018B
:100C40001A3033263A2627262E2E0030282E013041
:100C5000C6000C30C500582E01302F2E0430C600BF
:100C60000A30C500582E1F39C700C800C900CA0085
:100C7000C31708003F26C308031D3A2E0800431B74
:100C8000522E430803390319C313C30A4311C50085
:100C9000473E84000008F3009120F31B8038C60013
:100CA000C50A582E4313440DC40D0318272E252EB4
:100CB000851005110230F5004508F3000830F600F4
:100CC000F30D031C05100318051400008514000023
:100CD0008510F60B602E4608F50B5D2E05150800F5
:100CE0008D27722E8126473084000330F3000008E0
:100CF0007F39031D08001F308004840AF30B772E10
:100D0000080084008030C705000E0F39C70480300A
:100D1000C80500080F39C804040A84008030C905DA
:100D2000000E0F39C9048030CA0500080F39CA0403
:100D3000C3170800F300473084000430F50073083F
:100D4000C9208000F30A840AF50B9F2EC317080000
:100D5000AC0A2C088B23031DB02EAC01AD0AA82EC3
:100D6000840A801B092F001E382F0008F30003306F
:100D7000F400840A0008A4002D18F72E840A7308D2
:100D80006B283F30A5000008A600840A801EA61725
:100D9000801AA613F40AF52E0008A500FE3E031CD7
:100DA000E92EA600A5010310A60DA50DA60DA50D03
:100DB000A60DA50DA602031CA503A60DA50DA60D47
:100DC000A50DA60DA50D0430A5070310A50C03184D
:100DD0002516840A801AA512801EA5162517F31C55
:100DE000F52E001E2512001A251602301B2FAD18F5
:100DF000012F0230840700081F398038A500023017
:100E00001B2F0530840700080F39B038A500FF30CC
:100E10001B2F0530F400F103710807390319801303
:100E2000840A0008A4003408A5003508A600360886
:100E3000A70004301B2F8407800803192C2F2708D4
:100E4000A8002608A7002508A600240DA500000C70
:100E5000A50CC038A400F40A7408622FAB00A21FCE
:100E60002F2FA401A50103306227AB0B2F2F080001
:100E70000130AB00A21F3A2FFF30A4000030A500C4
:100E800003306227AB0B3A2F0800AB00A21F462F9E
:100E90000030A4007130A50003306227AB0B462F51
:100EA0000800AB00F011861DF015A21F532F340867
:100EB000A4003508A5003608A60004306227AB0B55
:100EC000532F0800A21F00280B12A200FE3EF300C1
:100ED0002430A10084000008840A0006840AF30B71
:100EE0006D2F80000B1608008400000E0F39F800EB
:100EF000F701AF2700080F39F8070318F70AAF27E3
:100F0000840A000E0F39F8070318F70AAF27000804
:100F10000F39F8070318F70A08000E30F500FA0138
:100F2000F9010310F80DF70DF80DF70DF80DF70D99
:100F3000FA0DF90DF50B9E2F793008007A30A327B2
:100F40007930A327962F840003300007F300F319AC
:100F5000800030300007F300F31B800008007808A1
:100F6000F3007708F4000310F80DF70D0310F80DE7
:100F7000F70D7308F8070318F70A7408F70703104A
:100F8000F80DF70D0800013083168100831206303A
:100F900081004030850007309F008316A030850017
:100FA00083128601831681130117FB3086008C01A2
:100FB000980118150E309900831298019701053099
:100FC00097000C11013090002030840080018417BC
:100FD00080018413831780018313840A841FE62F02
:040FE0000B17CF28F4
:02400E00433F2E
:104200000100000000004B00000000000000000062
:104210000F00160012001200050019000000170020
:104220000A000D000D00130017000A0009000E001F
:1042300017001300140009000000170005001F00FC
:104240000D00110013001F00130015001E001F00B9
:104250001E000100020008001E001F0002000800EE
:104260000000010000000000000000004D004200BE
:1042700024005200650076006900730069006F0039
:104280006E003A00200031002E003400370020007C
:1042900024000000FF00FF00FF00FF00FF00FF0000
:1042A000FF00FF00FF00FF00FF00FF00FF00FF0016
:1042B000FF00FF00FF00FF00FF00FF00FF00FF0006
:1042C000FF00FF00FF00FF00FF00FF00FF00FF00F6
:1042D000FF00FF00FF00FF00FF00FF00FF00FF00E6
:1042E000FF00FF00FF00FF00FF00FF00FF00FF00D6
:1042F000FF00FF00FF00FF00FF00FF00FF00FF00C6
:00000001FF
